:100000000C9436010C94A50A0C947E0A0C945E01A3
:100010000C945E010C94710C0C945E010C94430CD6
:100020000C94B60C0C945E010C945E010C945E0171
:100030000C945E010C945E010C945E010C945E01C4
:100040000C94340A0C945E010C94F20A0C94CC0AC1
:100050000C945E010C945E010C945E010C945E01A4
:100060000C94240B0C945E016803180172681880CC
:10007000234020034C69676874734F4E04034F4E4E
:10008000042020202020BE5004B03B805F50046834
:100090003B0205680576380A01285004683B282F82
:1000A0006805183802004F680576380A00295004A0
:1000B000683B212650046832101E50046832111F1C
:1000C000C004BF1103696804800200EE8003680168
:1000D000EA1804FF0200E16804C00200AEC0036831
:1000E00001AA681880234020035553426175646952
:1000F0006F04032020042020202020A168188023E2
:10010000402003425420417564696F040320200499
:100110002020202020F36818802340200320415510
:100120005820492F5004032020042020202020E9BB
:10013000681880234020034C6F6E677761766504F2
:10014000032020042020202020BC68188023402089
:10015000034D2E20576176652004032020042020C3
:10016000202020D568188023402003464D20626E51
:1001700064203204032020042020202020C268189C
:100180008023402003464D20626E6420310403200A
:1001900020042020202020C1681880234020034410
:1001A000414220626E64330403202004202020207A
:1001B00020AF6818802340200344414220626E64CF
:1001C0003204032020042020202020AE6818802341
:1001D00040200344414220626E6431040320200425
:1001E0002020202020AD6805183803004E680576D1
:1001F00038030020180A68390209003F000101771E
:100200006805183801004C6804BF0201D0000000E6
:1002100000240027002A0000000000250028002BF1
:1002200000000000080002010000030407000000B5
:100230000000000000000000002300260029000448
:10024000040404040404040202020202020303037D
:100250000303030102040810204080010204081077
:1002600020010204081020008E0D051311241FBE6A
:10027000CFEFD8E0DEBFCDBF24E0A2E7B1E001C000
:100280001D92A53BB207E1F711E0A0E0B1E0E0E28A
:10029000F9E202C005900D92A237B107D9F711E03B
:1002A000C5E3D1E004C02197FE010E944813C43386
:1002B000D107C9F70E946D0E0C9483140C940000B2
:1002C000833081F028F4813099F08230A9F00895CC
:1002D0008730A9F08830C9F08430B1F48091800073
:1002E0008F7D03C0809180008F7780938000089578
:1002F00084B58F7784BD089584B58F7DFBCF8091C1
:10030000B0008F778093B00008958091B0008F7D0A
:10031000F9CFCF93DF93282F30E0F901EF5DFD4F48
:100320008491F901ED5AFD4FD491F901E15CFD4F43
:10033000C491CC23A1F081110E946001EC2FF0E068
:10034000EE0FFF1FEB5CFD4FA591B491EC91ED23F7
:1003500081E090E009F480E0DF91CF91089580E0A2
:1003600090E0FACF1F93CF93DF93282F30E0F9016D
:10037000EF5DFD4F8491F901ED5AFD4FD491F901E4
:10038000E15CFD4FC491CC23A9F0162F81110E948E
:100390006001EC2FF0E0EE0FFF1FE95EFD4FA5912D
:1003A000B4918FB7F894EC91111108C0D095DE2369
:1003B000DC938FBFDF91CF911F910895DE2BF8CF93
:1003C000CF93DF9390E0FC01ED5AFD4F2491815CC7
:1003D0009D4FFC0184918823C9F090E0880F991FFC
:1003E000FC01E35FFD4FA591B491FC01E95EFD4F77
:1003F000C591D49161110DC09FB7F8948C9120954F
:1004000082238C938881282328839FBFDF91CF91FB
:100410000895623051F49FB7F8943C91822F8095F3
:1004200083238C93E8812E2BEFCF8FB7F894EC9138
:100430002E2B2C938FBFEACF3FB7F89480913A02CE
:1004400090913B02A0913C02B0913D0226B5A89B41
:1004500005C02F3F19F00196A11DB11D3FBFBA2F56
:10046000A92F982F8827BC01CD01620F711D811D16
:10047000911D42E0660F771F881F991F4A95D1F79B
:1004800008952FB7F89460913602709137028091E9
:100490003802909139022FBF089508950895089564
:1004A0000895AF92BF92CF92DF92EF92FF920F9397
:1004B0001F93CF93DF936C017B018B01040F151FFA
:1004C000EB015E01AE18BF08C017D10759F0699162
:1004D000D601ED91FC910190F081E02DC6010995C6
:1004E000892B79F7C501DF91CF911F910F91FF9073
:1004F000EF90DF90CF90BF90AF900895FC01538DA7
:10050000448D252F30E0842F90E0821B930B5417ED
:1005100010F0CF96089501970895FC01918D828D7A
:10052000981761F0A28DAE0FBF2FB11D5D968C9113
:10053000928D9F5F9F73928F90E008958FEF9FEF52
:100540000895FC01918D828D981731F0828DE80F0E
:10055000F11D858D90E008958FEF9FEF0895FC01C8
:10056000918D228D892F90E0805C9F4F821B910995
:100570008F73992708958EE392E00E94AF0221E0E5
:10058000892B09F420E0822F089580E090E0892BE8
:1005900029F00E94BB0281110C9400000895FC0117
:1005A000A48DA80FB92FB11DA35ABF4F2C91848DD4
:1005B00090E001968F739927848FA689B7892C9331
:1005C000A089B1898C91837080648C93938D848D84
:1005D000981306C00288F389E02D80818F7D808387
:1005E0000895EF92FF920F931F93CF93DF93EC0147
:1005F00081E0888F9B8D8C8D98131AC0E889F989CA
:10060000808185FF15C09FB7F894EE89FF896083CC
:10061000E889F98980818370806480839FBF81E04D
:1006200090E0DF91CF911F910F91FF90EF9008958F
:10063000F62E0B8D10E00F5F1F4F0F731127E02E6A
:100640008C8D8E110CC00FB607FCFACFE889F989A2
:10065000808185FFF5CFCE010E94CF02F1CFEB8DD7
:10066000EC0FFD2FF11DE35AFF4FF0829FB7F89476
:100670000B8FEA89FB8980818062CFCFCF93DF9394
:10068000EC01888D8823B9F0AA89BB89E889F989AA
:100690008C9185FD03C0808186FD0DC00FB607FCDF
:1006A000F7CF8C9185FFF2CF808185FFEDCFCE0112
:1006B0000E94CF02E9CFDF91CF9108952091BA0136
:1006C000260F3327331F21323105ECF42091090224
:1006D000FC0190E080E0243069F082E00895A09170
:1006E000BA012191AC0146565E4FA40FB52FB11D42
:1006F0002C930196861798F38091BA01680F609346
:10070000BA0180E0089581E008951092090281E025
:10071000809308021092E30161E082E10E94B2013D
:1007200061E083E10E94B201E9EBF0E080818E7F1D
:10073000808380818D7F808388E48093B80085E406
:100740008093BC000895CF93DF9391E0909399013B
:100750008823B9F0C091B800D091BA008091BC0054
:100760008A7B8093BC0060E082E10E94B20160E07D
:1007700083E10E94B2010E948503D093BA00C09326
:10078000B800DF91CF9108950895E091E201809142
:10079000E101E81730F4F0E0E758FE4F808190E087
:1007A00008958FEF9FEF08959091E2018091E1010C
:1007B0002FEF3FEF981748F4E92FF0E0E758FE4F8E
:1007C000208130E09F5F9093E201C90108958091FC
:1007D000E1019091E201891B990B0895CF92DF927C
:1007E000EF92FF920F931F93CF93DF937C01CB0186
:1007F0008A0120910F02222389F0EB016B01C40EC4
:10080000D51ECC15DD0569F06991D701ED91FC91FC
:100810000190F081E02DC7010995F3CF642F0E946C
:100820005E03C801DF91CF911F910F91FF90EF9070
:10083000DF90CF900895CF93DF931F92CDB7DEB7AF
:10084000698320910F022223F9F020913202203295
:1008500058F021E030E0FC013383228390E080E017
:100860000F90DF91CF91089580911002E82FF0E072
:10087000EF5EFD4F998190838F5F8093100280938C
:10088000320281E090E0ECCF61E0CE0101960E945F
:100890005E03F7CF90E080E00895FC0184819581AC
:1008A000228133812817390771F0860F971F6081E5
:1008B00071810E9434130680F781E02DE80FF91F43
:1008C000808190E008958FEF9FEF0895FC0184816F
:1008D0009581228133812817390741F0860F971FB0
:1008E000608171810E943413958384830895FC0193
:1008F000462F22813381C9010196608171810E9456
:100900003413648175818617970781F0A681B781BA
:10091000A20FB31F4C9382819381019660817181F4
:100920000E9434139383828380E008958FEF0895AB
:10093000EF92FF920F931F93CF93DF937C01062FCB
:1009400010E0B80181EA94E00E947704D0E0C0E0B2
:10095000C017D10758F4F701EC0FFD1F649170E048
:1009600081EA94E00E9477042196F2CFDF91CF9143
:100970001F910F91FF90EF900895CF93DF93FC01AB
:10098000C281D38184819581C817D907C9F0A68116
:10099000B781A80FB91F2C910196608171810E94C7
:1009A0003413C817D90739F095838483822F90E0D8
:1009B000DF91CF9108951582148213821282F6CFAF
:1009C0008FEF9FEFF5CFFC0160817181848195816C
:1009D0009B01281B390B82819381820F931F0E94F8
:1009E00034130895DC01ED91FC910190F081E02D2C
:1009F0000994809178018823B9F080917701882348
:100A000099F06CE084EF91E00E94980467E08DEE2D
:100A100091E00E94980467E086EE91E00E949804BD
:100A200061E08AE00C94B20160E08AE00E94B201C9
:100A300067E080E092E00C9498048F929F92AF92CE
:100A4000BF92CF92DF92EF92FF924B015C010E9426
:100A50001C026B017C0124E0C21AD108E108F108F4
:100A60000E941C026C197D098E099F096815790581
:100A70008A059B05A8F3FF90EF90DF90CF90BF9081
:100A8000AF909F908F9008958091DA03882319F09A
:100A900060E00C94B2012D980895882349F080916C
:100AA000DA03882319F061E00C94B2012D9A0895BD
:100AB0000C944405CF93DF93EC018091DB038230EB
:100AC00019F481E00E944D05299ABE0190E080E072
:100AD0000E941D0529988091DB03823031F40E9429
:100AE0004405DF91CF910C944405DF91CF91089597
:100AF0008F929F92AF92BF92CF92DF92EF92FF922E
:100B0000CF934B015C01219A8FEF88169806A806B7
:100B1000B806C1F4219A80E093E20E945A0560EC85
:100B200078E080E090E00E941D0580E392E0CF91A4
:100B3000FF90EF90DF90CF90BF90AF909F908F90FD
:100B40000C945A0580E093E20E945A0560E871E136
:100B500080E090E00E941D05C0E2C12CD12CE12C68
:100B600090E8F92ED501C4018C219D21AE21BF2131
:100B7000892B8A2B8B2B89F080E392E00E945A0507
:100B800060E976E080E090E00E941D05F694E7942D
:100B9000D794C794C15031F7C8CF80E392E00E9448
:100BA0005A0560E372E080E090E0EECFCF9329E554
:100BB00034E0F90101900020E9F79F012A55344003
:100BC000C091540433274C2F50E0BA016150710991
:100BD000261B370B30934F0420934E04682F70E090
:100BE000675A7B4F86E191E00E9473148091160151
:100BF000803219F486E880931601CB5FC09311010F
:100C0000EC2FF0E0319620E090E0A92FB0E0A05F5B
:100C1000BE4F4C9124279F5FC917B8F7E05FFE4F86
:100C200020836091110170E06E5F7F4F89EA94E04C
:100C30000E947704C0E02C2F30E08091110190E0F9
:100C40000196821793075CF0205F3E4FF9016081A7
:100C500070E089EA94E00E947704CF5FECCFCF91F7
:100C6000089585ED8093BC0080910B0290910C0259
:100C7000A0910D02B0910E020796A11DB11D23E0B7
:100C8000B695A795979587952A95D1F72091BC00A1
:100C900024FD03C010920902089540910B02509167
:100CA0000C0260910D0270910E02452B462B472BD2
:100CB00069F30097A105B10541F02AE22A95F1F701
:100CC00000C00197A109B109E1CF80910A020C94FB
:100CD000A303FC0186819781009711F00C94EA131D
:100CE00008951F93CF93DF93EC01162F0E941E13DC
:100CF000181739F0612FCE01DF91CF911F910C941D
:100D00002613DF91CF911F9108950C941E13CF935A
:100D1000DF9390E080E00E948506C82FD0E0D0935A
:100D20000B01C0930A018AE090E00E948506282FFB
:100D300030E030930901209308012197A9F48150F4
:100D4000873090F4E82FF0E0E755F94F6AE10C9412
:100D50004813B006C006C306C606C906CC06CF06B1
:100D60008CEC91E00E9498048AE090E00E94850655
:100D700090E09093090180930801DF91CF9108954D
:100D800082EB91E0EFCF88E991E0ECCF8EE791E044
:100D9000E9CF84E691E0E6CF8AE491E0E3CF80E317
:100DA00091E0E0CF90E080E00E948506282F30E0BF
:100DB00030930701209306018330D1F028F481306D
:100DC00041F0823061F008958430D1F08730E9F04D
:100DD0000895109277010E94F9040C9487061092EE
:100DE00077010E94F9046AE182EE90E00C94980485
:100DF000109277010E94F9046AE186E191E0F6CF52
:100E00006AE18CEF90E00E949804109277010C94B4
:100E1000F9048F929F92AF92BF92CF92DF92EF929E
:100E2000FF920F931F93CF93DF93CDB7DEB76897F1
:100E30000FB6F894DEBF0FBECDBF7C01FC01008170
:100E4000C280D38016810E944102809072019090EE
:100E50007301A0907401B09075019B01AC01281939
:100E600039094A095B0949015A0130E1831637E221
:100E70009306A104B10468F060937201709373014A
:100E8000809374019093750165E088E690E00E947C
:100E9000980445E050E06DED70E0C7010E94111329
:100EA000892B29F466E087ED90E00E94980446E0E3
:100EB00050E061ED70E0C7010E941113892B19F415
:100EC00081E0809378018091340281110AC066E04C
:100ED00087E092E00E9498040E94D20681E080930D
:100EE000340245E050E06CEC70E0C7010E94111341
:100EF000892B29F466E086EC90E00E94980445E096
:100F000050E060EC70E0C7010E941113892B11F4CE
:100F10000E94D206003809F073C24FEBC41273C2AC
:100F200058E1D51270C261E081E10E94B201809166
:100F30007601811105C00E94D20681E0809376017E
:100F400068960FB6F894DEBF0FBECDBFDF91CF918C
:100F50001F910F91FF90EF90DF90CF90BF90AF90D7
:100F60009F908F900895153009F487C0163041F78F
:100F700066E08AE990E00E949804809177018823D6
:100F800009F4B4C080917801882309F4AFC067E008
:100F900083E990E08CC0193009F4E1C008F4ABC0DB
:100FA0001A3009F48EC165E77AE88EE491E61B30C9
:100FB00009F446C2C5CF183209F406C248F5133207
:100FC00009F4CAC190F41E3009F0BACF61E08AE09A
:100FD0000E94B2018CE00E948901892B09F4B4C1FE
:100FE00060E08CE00E94B201A3C0163209F4DFC1B8
:100FF000173209F0A5CF80917701882321F08091E5
:101000007801811156C06FE070EF8EE491E618C24E
:101010001C3209F4A6C158F4193209F4ECC16FE589
:1010200070EA8EE491E61B3209F40AC289CF1D32C0
:1010300009F49CC11E3409F083CF60E08AE0689611
:101040000FB6F894DEBF0FBECDBFDF91CF911F91D9
:101050000F91FF90EF90DF90CF90BF90AF909F9057
:101060008F900C94B20166E08AEB90E00E949804A5
:1010700067ED78E28EE491E6E3C166E084EB90E010
:101080000E94980467E578EA8EE491E6D9C166E0AB
:101090008EEA90E00E9498048091770167E08823AF
:1010A000E1F0809178018823C1F087EA90E00E9406
:1010B000980468960FB6F894DEBF0FBECDBFDF91DF
:1010C000CF911F910F91FF90EF90DF90CF90BF9045
:1010D000AF909F908F900C94F90480EA90E00E946A
:1010E000980467EB78E48EE491E6AAC167E378ECB4
:1010F0008EE491E6A5C166E08DE890E00E94980438
:101100006FEA70E58EE491E60E9478058091060111
:1011100090910701019685309105F4F490930701B1
:10112000809306016091060190E080E00E947106C4
:1011300068960FB6F894DEBF0FBECDBFDF91CF919A
:101140001F910F91FF90EF90DF90CF90BF90AF90E5
:101150009F908F900C94D20681E090E0DFCF90E0DA
:1011600080E00E948506E82EF12CF0920B01E092BF
:101170000A0181E0E816F10409F067C06FE470EB42
:101180008EE491E60E94780587E090E09093050157
:1011900080930401809102019091030101968830AF
:1011A000910534F59093030180930201609102014F
:1011B0008BE090E00E9471068BE090E00E94850633
:1011C000282F30E0309303012093020181508730B3
:1011D00008F0B6CEE82FF0E0EF50F74F6AE10C943C
:1011E0004813FD081309160919091C091F092209CA
:1011F000F0920301E0920201D9CF8CEC91E0689665
:101200000FB6F894DEBF0FBECDBFDF91CF911F9117
:101210000F91FF90EF90DF90CF90BF90AF909F9095
:101220008F900C94980482EB91E0E9CF88E991E0EB
:10123000E6CF8EE791E0E3CF84E691E0E0CF8AE469
:1012400091E0DDCF80E391E0DACF90E080E00E9492
:10125000850690E090930B0180930A01029709F0B4
:101260006FCE809108019091090101969093090138
:101270008093080120910401309105012817390756
:1012800034F481E090E0909309018093080160912B
:1012900008018AE090E00E94710668960FB6F89403
:1012A000DEBF0FBECDBFDF91CF911F910F91FF9099
:1012B000EF90DF90CF90BF90AF909F908F900C9465
:1012C0008706809100019091010101968630910579
:1012D00064F590930101809300016091000188E220
:1012E00090E00E94710688E290E00E94850690E0FE
:1012F000909301018093000128E1E6E3F1E0DE0133
:10130000119601900D922A95E1F7880F991F880F89
:10131000991FE1E0F0E0EC0FFD1F8E0F9F1FFC0115
:1013200060817181828193818BC010920101109242
:101330000001D3CF66E087E890E00E94980465E959
:101340007AE68EE491E67CC061E08CE00E94B20116
:101350006AE18DE690E053CF6FE170EE8EE491E6A6
:101360006FC065EC7AE38EE491E66AC061E090E0DC
:1013700080E00E94710661E08AE090E00E947106C0
:1013800061E08BE090E00E94710660E08EE190E009
:101390000E94710660E088E290E00E94710660E0C1
:1013A0008CE890E00E9471060E94D20676CF809170
:1013B0007701882321F08091780181117ACE6FE83E
:1013C00070E78EE491E63CC062E090E080E06896D1
:1013D0000FB6F894DEBF0FBECDBFDF91CF911F9146
:1013E0000F91FF90EF90DF90CF90BF90AF909F90C4
:1013F0008F900C9471066FE470EB8EE491E620C040
:10140000003C09F09DCDF1E3DF129ACD61E085E06B
:101410000E94B2011C3009F48DCF08F0CCCD1730FA
:1014200009F435CE08F0B7CD143009F41CCE08F01D
:101430009ACD67E978E68EE491E6133009F080CD25
:1014400068960FB6F894DEBF0FBECDBFDF91CF9187
:101450001F910F91FF90EF90DF90CF90BF90AF90D2
:101460009F908F900C9478051F920F920FB60F9259
:1014700011242F933F938F939F93AF93BF938091AA
:10148000360290913702A0913802B0913902309122
:10149000350223E0230F2D3758F50196A11DB11D0C
:1014A000209335028093360290933702A09338023E
:1014B000B093390280913A0290913B02A0913C0294
:1014C000B0913D020196A11DB11D80933A02909307
:1014D0003B02A0933C02B0933D02BF91AF919F911C
:1014E0008F913F912F910F900FBE0F901F901895E5
:1014F00026E8230F0296A11DB11DD2CF1F920F9295
:101500000FB60F9211242F933F934F935F936F93D6
:101510007F938F939F93AF93BF93EF93FF93E0914C
:101520000E01F0910F010995FF91EF91BF91AF91DD
:101530009F918F917F916F915F914F913F912F91EB
:101540000F900FBE0F901F9018951F920F920FB61D
:101550000F9211242F933F934F935F936F937F9339
:101560008F939F93AF93BF93EF93FF93E0910C0101
:10157000F0910D010995FF91EF91BF91AF919F916E
:101580008F917F916F915F914F913F912F910F902C
:101590000FBE0F901F9018951F920F920FB60F92CB
:1015A00011242F933F934F935F936F937F938F9368
:1015B0009F93AF93BF93EF93FF938EE392E00E94CC
:1015C000CF02FF91EF91BF91AF919F918F917F914A
:1015D0006F915F914F913F912F910F900FBE0F90A0
:1015E0001F9018951F920F920FB60F9211242F93F0
:1015F0008F939F93EF93FF93E0914E02F0914F02F0
:101600008081E0915402F091550282FD1BC09081CF
:10161000809157028F5F8F7320915802821741F09B
:10162000E0915702F0E0E25CFD4F958F8093570206
:10163000FF91EF919F918F912F910F900FBE0F907F
:101640001F9018958081F4CF1F920F920FB60F92C2
:1016500011242F933F934F935F936F937F938F93B7
:101660009F93AF93BF93EF93FF938091B900887FCF
:10167000803609F44AC0F0F5883209F4A7C018F59D
:10168000803109F49BC0B8F4882309F4F9C088308C
:1016900009F494C0FF91EF91BF91AF919F918F9109
:1016A0007F916F915F914F913F912F910F900FBE5E
:1016B0000F901F901895883109F488C0803251F737
:1016C0008093070214C0803409F49DC040F4803335
:1016D000B9F38833F9F68093070285ECB0C0803502
:1016E00009F485C0883509F496C0883499F60E94BB
:1016F0003106D0CF883909F48CC038F5883729F005
:1017000050F4883611F0803729F683E0809309027F
:101710001092DC0157C0883809F47BC0803919F079
:10172000803809F0B7CF8091DC01803208F071C0B9
:10173000E091DC0181E08E0F8093DC018091BB00A1
:10174000F0E0E454FE4F80833DC0803B39F0E0F48C
:10175000803A09F479C0883A09F09CCF84E08093FC
:1017600009021092BB011092BA01E091DF01F091E1
:10177000E00109958091BA0181110FC081E0809349
:10178000BA0110929A0109C0803C09F4A6CF883CA6
:1017900009F4A3CF883B09F07DCFE091BB0181E044
:1017A0008E0F8093BB01F0E0E656FE4F8081809360
:1017B000BB009091BB018091BA0129C08091E401E6
:1017C0008093BB0085EC8093BC0064CF90910602AF
:1017D00080910502981758F5E091060281E08E0F7E
:1017E00080930602F0E0EB51FE4F8081E9CFE0915B
:1017F000060281E08E0F809306028091BB00F0E02C
:10180000EB51FE4F8083909106028091050298175C
:10181000C8F285E8D8CFE091060281E08E0F809370
:1018200006028091BB00F0E0EB51FE4F8083809177
:10183000080281115CCF81E08093E30184EA809308
:10184000BC001092090226CF85EC8093BC00109258
:1018500009028091DC01803230F4E091DC01F0E09B
:10186000E454FE4F10826091DC0170E0E091DD01F4
:10187000F091DE018CEB91E009951092DC010ACF2A
:101880001092070234CF1F920F920FB60F921124BD
:101890002F933F934F935F936F937F938F939F9378
:1018A000AF93BF93EF93FF9381E08093330260E0A7
:1018B0008DE00E94B201E1EBF0E08081887F8083BF
:1018C000FF91EF91BF91AF919F918F917F916F9118
:1018D0005F914F913F912F910F900FBE0F901F90EE
:1018E00018951F920F920FB60F9211242F933F93CA
:1018F0004F935F936F937F938F939F93AF93BF9318
:10190000EF93FF9380E00E9489010197D9F481E071
:101910000E9489010197B1F48091B10087608093A2
:10192000B100FF91EF91BF91AF919F918F917F9106
:101930006F915F914F913F912F910F900FBE0F903C
:101940001F90189580E00E948901892B51F781E052
:101950000E948901019729F71092330261E08DE01E
:101960000E94B2018091B100887FD9CF1F920F925F
:101970000FB60F9211242F933F934F935F936F9362
:101980007F938F939F93AF93BF93CF93EF93FF93E7
:10199000E091F102F091F202C0818091F302C8233C
:1019A0008091F4029091F502019649F08091F40241
:1019B0009091F50201969093F5028093F402809144
:1019C000EF0281111DC0C1116EC08091F40290918F
:1019D000F502813A910578F01092F8028091F402B4
:1019E0009091F5029093FB028093FA0281E080933C
:1019F000F9028093EF021092F5021092F40253C0A4
:101A00008091EF028130A9F4CC2309F44CC0E0911D
:101A1000F9028E0F8093F9028091F4029091F50201
:101A2000F0E0EE0FFF1FE151FD4F9487838782E0C6
:101A3000E0CF8091EF02823009F04FC0C11122C087
:101A4000E091F90281E0E03768F08093F80283E0EA
:101A50008093EF02E091F602F091F702309759F28D
:101A60000995C9CF8E0F8093F9028091F40290916D
:101A7000F502F0E0EE0FFF1FE151FD4F94878387E1
:101A800081E0B7CF8091F4029091F502813A9105FF
:101A900050F083E08093EF02E091F602F091F702BC
:101AA000309709F009958091DB03813021F4C11151
:101AB00080E00E944D05FF91EF91CF91BF91AF91D2
:101AC0009F918F917F916F915F914F913F912F9156
:101AD0000F900FBE0F901F9018958091EF028330EA
:101AE00011F7C111E0CF87CF0F931F93CF93DF93EF
:101AF000EC018B01798368831D821C821B821A8210
:101B0000CB010E944E139F838E83A80170E060E09A
:101B1000DF91CF911F910F910C947C14CF93DF93A1
:101B2000EEE3F2E01382128288EE93E0A0E0B0E0F0
:101B300084839583A683B78322E531E031832083B4
:101B400025EC30E03587248724EC30E03787268782
:101B500020EC30E0318B208B21EC30E0338B228B7A
:101B600022EC30E0358B248B26EC30E0378B268B53
:101B7000118E128E138E148EEBEDF2E01382128210
:101B800084839583A683B78384E691E091838083E1
:101B90000E9441026093EB027093EC028093ED028D
:101BA0009093EE020E9441026093E7027093E80274
:101BB0008093E9029093EA0260E870E089E994E09A
:101BC0000E94740D60E470E081EA94E00E94740D5C
:101BD00060E470E089EA94E00E94740DEFEEF2E0B8
:101BE000F0930304E0930204118281E0848389E28C
:101BF00090E09383828350981092DA03CFE0D4E090
:101C00001CAA0E9441026093EB027093EC02809345
:101C1000ED029093EE020E9441026093E7027093FE
:101C2000E8028093E9029093EA0219861A861B86DD
:101C300018861F821E821D8262E080E00E94E00101
:101C400061E084E00E94E00161E084E00E94B20172
:101C5000E0EBF0E010821092B1008DE98093B300C8
:101C6000808182608083E0E7F0E080818260808311
:101C7000E8E6F0E0808184608083EDE6F0E080813A
:101C80008160808319821A8280ED97E09AAF89AFD4
:101C900088EE93E09CAF8BAF88EC90E09EAF8DAF69
:101CA00082E08093550410924F0410924E048BE012
:101CB00080935404109256041092570410925804C2
:101CC0000E94410260935004709351048093520427
:101CD00090935304DF91CF910895789484B58260F6
:101CE00084BD84B5816084BD85B5826085BD85B5C0
:101CF000816085BD80916E00816080936E0010923E
:101D000081008091810082608093810080918100B8
:101D10008160809381008091800081608093800049
:101D20008091B10084608093B1008091B0008160A7
:101D30008093B00080917A00846080937A008091D3
:101D40007A00826080937A0080917A00816080932B
:101D50007A0080917A00806880937A001092C100A6
:101D600061E085E00E94E00161E086E00E94E00120
:101D700060E08AE00E94E00161E08BE00E94E00107
:101D800061E08CE00E94E00162E084E10E94E001F9
:101D900061E08DE00E94E001E0914E02F0914F027F
:101DA00082E08083E0914A02F0914B021082E09140
:101DB0004C02F0914D0280E1808310925602E09136
:101DC0005202F091530286E08083E0915002F0913C
:101DD0005102808180618083E0915002F091510234
:101DE000808188608083E0915002F091510280816F
:101DF00080688083E0915002F091510280818F7D54
:101E0000808361E085E00E94B2011092E2011092AD
:101E1000E10110921002109232020E9485038EE4BA
:101E200092E09093E0018093DF018FE492E0909341
:101E3000DE018093DD0181E080930F028FE28093C9
:101E400031026FE78BED92E00E941B04C0913202D9
:101E5000C13208F091C00E941C026B017C0180918C
:101E60000902811164C082E08093090281E08093BD
:101E700008028FEF8093070210920602C0930502BA
:101E8000A1E1B2E0E5EEF1E080E0C81323C11092D9
:101E9000E4018091E4018E658093E4018091E30187
:101EA000813009F01BC11092E3010E941C026B01FA
:101EB0007C018091E4018093BB0080910B029091A2
:101EC0000C02A0910D02B0910E02892B8A2B8B2B54
:101ED00099F00E941C0200910B0210910C022091BB
:101EE0000D0230910E026C197D098E099F090617AB
:101EF000170728073907E0F18091BC0083FDD9CF8F
:101F000085EC8093BC000E941C026B017C018091D7
:101F10000902823009F4E4C0809107028F3F61F129
:101F200080910702803241F18091070225C08091A3
:101F30000B0290910C02A0910D02B0910E02892B20
:101F40008A2B8B2B09F48BCF0E941C0200910B0271
:101F500010910C0220910D0230910E026C197D0936
:101F60008E099F09061717072807390708F077CF4A
:101F700080910A020E94A303109210021092320272
:101F800010920F028EE392E0909313048093120458
:101F9000E0914E02F0914F0292E09083E0914A026C
:101FA000F0914B021082E0914C02F0914D028FECC7
:101FB000808310925602E0915202F091530286E221
:101FC0008083E0915002F091510280818061808392
:101FD000E0915002F0915102808188608083E0910D
:101FE0005002F0915102808180688083E09150021C
:101FF000F091510280818F7D80832CED35E030930C
:1020000049042093480428EE33E030934B04209396
:102010004A0428EC30E030934D0420934C04909314
:10202000550489E097E0909347048093460461E06B
:102030008DE00E94E00192E0292E312CEE24E39401
:10204000F12C34E0C32ED12C8091340281112FC0A9
:102050000E941C024B015C0188EE482E83E0582E42
:10206000612C712C0E941C02681979098A099B094C
:10207000683E734081059105A8F321E0421A51089A
:102080006108710888EE880E83E0981EA11CB11CBF
:10209000411451046104710429F766E087E092E07D
:1020A0000E9498040E94D206B1E0B0933402E091FD
:1020B0001404F0911504E830F105B0F5EE59FF4E27
:1020C0000C94481392104D1163118611AF11C41175
:1020D000D811F9119D9191938F5FD7CE85EE11CFD5
:1020E00080910B0290910C02A0910D02B0910E0212
:1020F000892B8A2B8B2B09F40ACF0E941C0200919A
:102100000B0210910C0220910D0230910E026C19FD
:102110007D098E099F09061717072807390708F058
:10212000F6CE26CF10925604809133028823E1F038
:1021300089EA94E00E94E30418161906ACF489EACF
:1021400094E00E94BD04EC0180E00E9489010197A7
:1021500031F4B12CA12CC331D10508F470C1BE01FA
:1021600089EA94E00E94660480911204909113041D
:10217000DC01ED91FC910084F185E02D0995892B1E
:1021800081F08091120490911304DC01ED91FC9197
:102190000284F385E02D0995BC0189E994E00E9451
:1021A000770480911604909117048230910509F408
:1021B0009BC108F058C1009709F463C1019709F465
:1021C00075C1809133028823C9F181EA94E00E94AD
:1021D000E3041816190694F50E9441020091E702E3
:1021E0001091E8022091E9023091EA02601B710B24
:1021F000820B930B6A30710581059105F8F081EA35
:1022000094E00E94BD04EC0180E00E9489010197E6
:1022100031F4B12CA12CC132D1050CF4E2C1BE01C4
:1022200081EA94E00E9466040E9441026093E70202
:102230007093E8028093E9029093EA02809110047F
:10224000882371F00E94410260E084E00E94B201A4
:1022500070E060E080911204909113040E94F204F7
:102260000E94410261347F418105910548F08BE075
:102270000E948901019721F460E08BE00E94B20185
:1022800080E090E0892B09F4DFCE0E94BB02882316
:1022900009F4DACE0E940000D7CE109258041092B2
:1022A000570480E00E94D605309215042092140451
:1022B0000E94410260935004709351048093520431
:1022C0009093530431CF0E94410200915004109129
:1022D00051042091520430915304AB01BC01401BC6
:1022E000510B620B730B8091480490914904B0E04C
:1022F000A0E0481759076A077B0708F415CF83E069
:1023000090E090931504809314040ECF80915704AD
:1023100020914E0430914F048217130680F48F5F92
:10232000809357048091580491E0980F909358043B
:102330000E94D605D0921504C0921404B9CFA5E02E
:10234000B0E0B0931504A0931404109258041092B6
:102350005704809156048F5F80935604E5CE0E9407
:102360004102009150041091510420915204309187
:102370005304AB01BC01401B510B620B730B8091EA
:102380004C0490914D04B3CF909156048091550424
:10239000981738F486E090E0909315048093140425
:1023A00087CFA7E0B0E0B0931504A093140480CFCA
:1023B0000E94410200915004109151042091520456
:1023C00030915304AB01BC01401B510B620B730BEA
:1023D00080914A0490914B04B0E0A0E0481759075F
:1023E0006A077B0708F4A0CEF0921504E09214046B
:1023F0009BCE0E9441020091500410915104209103
:10240000520430915304AB01BC01401B510B620BD1
:10241000730B80914A0490914B04B0E0A0E0481700
:1024200059076A077B0708F47FCE1092580480E0B2
:102430000E94D605109215041092140475CE0091D6
:10244000120410911304CA15DB0509F48DCE89EA34
:1024500094E00E94BD04BC01C8010E94F204BFEFD9
:10246000AB1ABB0AECCF8330910509F477C061E069
:1024700070E0049709F0A5CE89E994E00E94660413
:10248000ABC089E994E00E94E304181619060CF029
:1024900098CE70E060E089E994E00E944D0480935A
:1024A0001804F0921704E09216048BCE89E994E0A8
:1024B0000E94E30402970CF484CE61E070E089E9A5
:1024C00094E00E944D04809319048350823228F4D2
:1024D000309217042092160474CE61E070E089E90E
:1024E00094E00E9466046DCE0091190410E058013A
:1024F000BFEFAB1ABB0A89E994E00E94E304A81677
:10250000B9060CF05ECE712CD0E0C0E0BE0189E9C6
:1025100094E00E944D04782621960C171D07B4F70D
:10252000B50189E994E00E944D047816190689F4F2
:102530000E9441026093EB027093EC028093ED02E3
:102540009093EE0283E090E090931704809316043A
:1025500038CED0921704C092160433CE809118045E
:10256000982F9F77903521F0982F9F7B903899F482
:10257000CFE0D4E09E012F50344021968091190481
:1025800090E0019682179307ECF089E994E00E94AD
:10259000BD048B87EFCF893759F3982F9D7F9836ED
:1025A00039F38F3329F3883119F3982F9F7D983CA5
:1025B000F9F26091190470E06E5F7F4F803B09F083
:1025C0005BCFD6CF91E090934304E0914604F09125
:1025D00047048BE194E009951092170410921604B9
:1025E000F0CDAC16BD060CF01FCE00911204109178
:1025F000130481EA94E00E94BD04BC01C8010E945A
:10260000F204AFEFAA1ABA0AECCF89EA94E00E946A
:10261000690681EA94E00E94690689E994E00C94D5
:102620006906FB01DC0104C08D910590801921F43D
:1026300041505040C8F7881B990B0895F999FECF77
:1026400092BD81BDF89A992780B50895262FF999F2
:10265000FECF1FBA92BD81BD20BD0FB6F894FA9A85
:10266000F99A0FBE01960895AA1BBB1B51E107C042
:10267000AA1FBB1FA617B70710F0A61BB70B881F12
:10268000991F5A95A9F780959095BC01CD010895A1
:10269000EE0FFF1F0590F491E02D09940F931F9307
:1026A000CF93DF938230910510F482E090E0E091C7
:1026B000B304F091B40430E020E0B0E0A0E0309743
:1026C00099F42115310509F44AC0281B390B24302F
:1026D0003105D8F58A819B816115710589F1FB016E
:1026E00093838283FE0111C0408151810281138155
:1026F00048175907E0F04817590799F4109761F007
:1027000012960C93129713961C933296CF01DF9179
:10271000CF911F910F9108950093B3041093B404C7
:10272000F4CF2115310551F04217530738F0A901B4
:10273000DB019A01BD01DF01F801C1CFEF01F9CF43
:102740009093B4048093B304CDCFFE01E20FF31F46
:10275000819391932250310939832883D7CF2091D7
:10276000B1043091B204232B41F420913201309115
:1027700033013093B2042093B104209130013091A1
:1027800031012115310541F42DB73EB74091340197
:1027900050913501241B350BE091B104F091B20446
:1027A000E217F307A0F42E1B3F0B2817390778F028
:1027B000AC014E5F5F4F2417350748F04E0F5F1F87
:1027C0005093B2044093B104819391939FCFF0E072
:1027D000E0E09CCFCF93DF930097E9F0FC013297C4
:1027E00013821282A091B304B091B404ED0130E0E1
:1027F00020E01097A1F420813181820F931F209156
:10280000B1043091B2042817390709F061C0F09380
:10281000B204E093B104DF91CF910895EA01CE179D
:10282000DF07E8F54A815B819E0141155105B1F74B
:10283000E901FB83EA8349915991C40FD51FEC1735
:10284000FD0761F4808191810296840F951FE90153
:1028500099838883828193819B838A83F0E0E0E07F
:1028600012968D919C9113970097B9F52D913C91FB
:102870001197CD010296820F931F2091B1043091E0
:10288000B2042817390739F6309751F51092B4047D
:102890001092B304B093B204A093B104BCCFD3831D
:1028A000C28340815181840F951FC817D90761F4F5
:1028B0004E5F5F4F88819981480F591F5183408334
:1028C0008A819B81938382832115310509F0B0CFE2
:1028D000F093B404E093B3049ECFFD01DC01C0CFBC
:1028E00013821282D7CFFB01DC0102C001900D924E
:1028F00041505040D8F70895DC0101C06D9341501C
:102900005040E0F7089511E0C5E3D1E004C0FE01B6
:102910000E9448132196C633D107C9F7F894FFCF18
:1029200001000100010001000100010050025002FD
:10293000C8008023423200000000000000000000B8
:102940000000000000000000000000000000000087
:102950000000B50480007D824E61BD424E613DC2E3
:102960004E61DD224E615DA24E619D624E610000AE
:102970000000F10251027E023E03AF028D02A1026D
:10298000000000001B04EE034A04C403E703D40361
:02299000C5037D
:00000001FF
